:10000000B528A60014200C080D040319B028AA2056
:1000100084132608800664000D280E288C0A031914
:100020008D0F0B288006B028FF3A84178005B02872
:100030008001840AFF3E031D1828B028890083161A
:10004000081483120808B028880083160815553054
:100050008900AA308900881488182C280811B02833
:100060008F018E00FF308E07031C8F07031CB02802
:1000700003308D00DF303E2032288D01E83E8C00B9
:100080008D09FC30031C47288C07031844288C0773
:1000900064008D0F44280C184D288C1C512800003A
:1000A0005128080003108C0D8D0DFF3E03185228B7
:1000B0000C08B0288E00023068288E0003306828B3
:1000C0008E00013068288E00063068288E000530CA
:1000D00094000F080D02031D6F280E080C02043057
:1000E00003180130031902301405031DFF30B02836
:1000F00091019001103092000D0D900D910D0E08A0
:1001000090020F08031C0F0F910203188E280E088F
:1001100090070F0803180F0F910703108C0D8D0D1A
:10012000920B7C280C08B028103094008D018C01B3
:10013000930C920C031CA2280E088C070F080318BE
:100140000F0F8D078D0C8C0C910C900C940B982834
:100150001008B0288C098D098C0A03198D0A080033
:100160008313031383126400080083161F30850075
:100170008601831286010C30840044301820061654
:1001800003308F00E8303120061203308F00E83052
:10019000312018301E20B20019301E20B3002E303E
:1001A0001E20C800132132088C0033088D008F01F7
:1001B00000306620031DEC2806160F3005059E0052
:1001C0009F011E088C001F088D008F0108305A20E7
:1001D000031DEB28DD280612412132088C0033086C
:1001E0008D008F0100306620031D06293A08103C5F
:1001F000B2003B08031C013E273CB30018308900C5
:10020000320824201930890033082420BA01BB01A8
:10021000FA3030200130C5001A301E20BC001B30DF
:100220001E20BD00E32A2E308900480824206400E7
:1002300003304802031C202944140330C80221293A
:100240004410CA01640008304A02031840294808D3
:100250009200930108308E008F0194209E001108B7
:100260009F004A089E0703189F0A1E081E20A00030
:10027000A1014A082A3E840020088000CA0F2229D2
:100280000800640001304802031C49290230BE0006
:100290004B290130BE001030BA002730BB000730B8
:1002A0003A05B400B50134082A3E840000088600EF
:1002B000143030206400051E5E2963293E08BA020E
:1002C000031CBB034F293408B8003508B9000800E7
:1002D0000508C9006400051E7329BA01BB01340872
:1002E000B8003508B9000F30C90564000130490273
:1002F000031C7C29B601B7016400430849020319B5
:100300008229BF014908C30049080F3C031C9C29EE
:1003100001308A00490882079D29B729C229CE29C0
:10032000DA290D2A0F2A9D29372A9D299D299D29E1
:100330001F2A9D299D293A2B682936088C003708E9
:100340008D0003308F00E8306620031DAF29640064
:10035000441CAD29003041048600C501B229B60A0B
:100360000319B70A03303020C414BF0168296400A0
:1003700001304502031CBD29492AC0016430C20076
:10038000A5236829640001304502031CC829B92A45
:100390000130C0006430C200A5236829BF0AC5012E
:1003A000FA30302064000C303F020318D829682945
:1003B000BF01B528BF0AC501323030206400C83003
:1003C0003F020318E42968292E301E20C800C80AFD
:1003D00064004808063C031DEE29C8012E30890040
:1003E000480824200130CA00013048079E009F01C0
:1003F0009F0D4A088C008D011F088F001E08602089
:10040000031D072AB422C8303020CA0FF429013056
:100410008F00F430312013216829C001112A0130E6
:10042000C000FA30C200C501640004303F02031866
:100430001B2ABF0A1D2A1430C200A52368296400A4
:100440000C303F020318292ABF0AFA3030206829ED
:10045000362A1830CA0064002F304A020318362AA0
:100460004A08890000302420CA0F2B2AB5286400CE
:1004700014303F020318402ABF0A1930302068297F
:1004800064000A3045020318462AC50AB422BF0197
:100490006829061601308F002C3031200508CA006B
:1004A00064004A08003C031D562A4E2A64004A088C
:1004B000013C03195E2A0612C5016829FA30302072
:1004C000CA010F300505CB0064004B08013C03193D
:1004D0006C2AC50106126829CA0AFA303020640065
:1004E00007304A020318752A612A023092009301EC
:1004F00045088E008F0194209E0011089F0018303F
:100500009E0703189F0A1E0889003A08242002301B
:100510009200930145088E008F0194209E001108DF
:100520009F0019309E0703189F0A1E0889003B0888
:1005300024200612C50103308F00E83031206829DD
:1005400001308F00F43031200130CA0064004A08C5
:100550004502031CB32A06167D30302006127D307A
:100560003020CA0FA62A08000616C830302006120E
:100570000800A02264004508003C031DC12A013088
:10058000C50002309200930145088E008F0194202F
:100590009E0011089F0018309E0703189F0A1E082E
:1005A0001E20BC0002309200930145088E008F018E
:1005B00094209E0011089F0019309E0703189F0A7F
:1005C0001E081E20BD0001303A079E003B0803189C
:1005D000013E9F003C088C003D088D001F088F00E5
:1005E0001E086620031DF52A302B01303A029E00BA
:1005F0000030031C013E3B029F003C088C003D087C
:100600008D001F088F001E086620031D082B302B4D
:100610003C088C003D088D003B088F003A0866209E
:10062000031D152BA022C50168293C088C003D083C
:100630008D003B088F003A085D20031D202BC00170
:100640003C088C003D088D003B088F003A08632071
:10065000031D2C2B0130C0001430C200A523E32A57
:10066000640001304802031C392BA022C50168290F
:100670003A2B082B2A3030200F300505CA001E30D7
:1006800030200F300505CB0064004A08003C031DF4
:10069000552B4B088C008D0105305520C1004108B9
:1006A0008604323030206829A52B1E3030204B08BC
:1006B0008C008D0104305520CB000F300505C9009A
:1006C0004908CB044B0892009301B4308E008F018F
:1006D00094209E0011089F001E088C001F088D00AA
:1006E000FF308E008F0178209E000D089F003C3067
:1006F0001E07C6003230302064004A08023C031D49
:10070000892B46088C008D010630840020300120A2
:10071000902B46088C008D0106308400403001206B
:100720000130CB00640006304B020318A42B0330C9
:1007300030200F300505C900640001304902031C58
:10074000A22B6829CB0F922B7C2B01304006BE00D8
:10075000640001304802031CBD2B40089200930145
:1007600002308E008F019420C0003E089200930159
:1007700002308E008F019420BE003E088C008D0157
:100780003B088F003A086320031DC72B68294008E7
:100790003A079E003B080318013E9F001E088C008C
:1007A0001F088D0033088F0032086320031DD92BEA
:1007B000682940083A079E003B080318013E9F0045
:1007C0003E081E02BA001F08031CFF3EBB003A0889
:1007D00038079E003B080318013E39079F00073089
:1007E0001E05B40000301F05B50034082A3E840001
:1007F00000089E001E0841048600420830200800C0
:02400E00F53F7C
:10420000010003000200060004000C000800090081
:104210000100010002000200040004000800080080
:1042200003000300060006000C000C000900090052
:10423000000000000000000000000000000000007E
:10424000000000000000000000000000000000006E
:0E425000000000000000000000000000000060
:00000001FF
